:1060000055C00000B7C00000B5C00000B3C000001C
:10601000B1C00000AFC00000ADC00000ABC00000C8
:10602000A9C00000A7C00000B8C50000A3C00000C0
:10603000A1C000009FC000009DC000009BC00000E8
:1060400099C0000097C0000095C0000093C00000F8
:1060500015C200008FC000008DC000008BC0000082
:1060600089C0000087C0000085C0000083C0000018
:1060700081C000007FC000007DC000007BC0000028
:1060800079C0000077C0000075C0000073C0000038
:1060900071C000006FC000006DC000006BC0000048
:1060A00069C0000067C0000065C0000011241FBE69
:1060B000CFEFDAE0DEBFCDBF89E0E3E0F0E0809330
:1060C000570084918E7F91F004B601FE0AC081E0F2
:1060D000209181013091820122343C4D19F080E001
:1060E00001C081E094B79D7F94BF11C004B603FE48
:1060F0000AC081E0209181013091820122343C4D1F
:1061000019F080E001C080E094B7977F94BF30E041
:1061100020E0F901459154918823B9F04F3F5F4F3A
:10612000A1F084B7877F84BF0FB6F894A8958091BB
:106130006000886180936000109260000FBE109232
:10614000820110928101F901099511E0A0E0B1E00E
:10615000E0ECFEE602C005900D92A436B107D9F737
:1061600021E0A4E6B1E001C01D92A138B207E1F739
:106170003CD1A4C645CF815098F09091F300209176
:10618000F200392F232B69F49091E8009B7F9093C4
:10619000E8009091E80092FDEECF9EB39111F9CF07
:1061A00008959091F100E7CFECE6F1E082819381D0
:1061B000582F492F848195819827892798275093B4
:1061C000670140936601909365018093640108958F
:1061D0001F93CF93DF9300D00F92CDB7DEB780919E
:1061E0006C01909176019923F1F1843039F5809119
:1061F0006D01811126C080916E018F3F11F5809154
:106200006D01833009F09DC081E08093750180911C
:106210006E01E0917201F0917301309709F476C03C
:106220008130D1F480917001909171019827892774
:10623000982790936A01809369010EC0853009F414
:10624000A4C08AE08093000183E080937401809170
:10625000EB0080628093EB000F900F900F90DF9126
:10626000CF911F910895843051F260F48130E1F0B4
:10627000833091F780916D01982F9D7F61F594DFB8
:1062800089E026C0853009F480C0863029F78091E6
:106290006D01833009F780916E018111DDCF80910E
:1062A0006F0180936801D8CF10916D011230A0F674
:1062B0007BDF11110CC0809166019091670123E092
:1062C000FC0120935700E89507B600FCFDCF85E060
:1062D00080930001C1CF813009F0BECFF0E0E0E053
:1062E00084918F3F69F010926801F0936701E09309
:1062F00066018AE08093000185E080937401ACCF51
:106300003196E11520E6F20759F7A6CF811111C0A9
:1063100082E49CED909382018093810188E19CE06E
:106320000FB6F894A895809360000FBE909360001C
:1063300093CF85919491019609F08ECF109201012F
:106340008BCF811189CF80916E018F3F09F084CF6F
:10635000F0E0E0E083E095E080935700E89507B631
:1063600000FCFDCF90935700E89507B600FCFDCFE9
:10637000E058FF4FE11520E6F20771F781E18093C5
:106380005700E8951092760167CF809102019091B5
:106390000301A091040189839A83AB83E0916E018C
:1063A00080916D01811109C0E33080F4EC0FFD2F65
:1063B000F11D818180936B014FCF813009F04CCF6B
:1063C000E13379F040F488E5E033A1F38AE080938B
:1063D000000188E092CFE03631F087E8E13651F3F2
:1063E000F5CF8EE1E7CF85E9E5CF84B7877F84BF1E
:1063F0000FB6F894A8958091600088618093600042
:10640000109260000FBE80E890E00FB6F894809381
:106410006100909361000FBEC1E0C5BF82E085BFFF
:106420009FD38AB1806F8AB98BB18F708BB9C093BB
:106430006F0083E0809381008BB18F7080618BB996
:10644000789480910101811117C0809175018111AB
:1064500013C033D38AB18F708AB98BB18F708BB967
:1064600010926F001092810081E085BF15BEE0910F
:106470006901F0916A010995FFD4E3CF8F9380E31E
:1064800089B98F9118957F928F929F92AF92BF9208
:10649000CF92DF92EF92FF920F931F93CF93DF93F0
:1064A000809179018F778132A9F480E389B9809155
:1064B0007F0190918001909373018093720180918C
:1064C0007A01833009F4B5C198F4813009F1823042
:1064D00009F41DC1DF91CF911F910F91FF90EF90B3
:1064E000DF90CF90BF90AF909F908F907F90089556
:1064F000853009F4C4C108F4BAC1863059F78091D7
:10650000E800877F8093E80082E08093000125C047
:106510008091E800877F8093E8008091750188234F
:1065200019F056DE109275018091720190917301FD
:10653000009729F580910001853051F48091720116
:1065400090917301892B09F041C082E08093000192
:106550008091E8008B7F8093E800DF91CF911F91BD
:106560000F91FF90EF90DF90CF90BF90AF909F90F2
:106570008F907F9085C22EB3222309F4ABCF209158
:10658000E80022FFF8CF2091F10020936C010197E1
:106590009093730180937201EDE6F1E09091F30026
:1065A0008091F200892B81F08091F100819380919C
:1065B000720190917301019790937301809372011E
:1065C00021E0E237F20751F703DEB4CF8AE1D3DDF1
:1065D0000091660110916701802F8F71CCDDC09111
:1065E0006401D09165012196C01BD10B20916D01F2
:1065F00021117DC0D695C795C80130916801A32FA0
:10660000B0E0480111E005E033E0732EAE014150E7
:106610005109CD2B79F4809164019091650190939B
:1066200067018093660181E180935700E89580E1DE
:10663000A2DD8ECF3091F3006091F200732F672BB3
:1066400069F1E091F1003091F1006E2F732FFC01A0
:106650000B0110935700E89511242F5F6C017D0109
:10666000F2E0CF0ED11CE11CF11CD701C601203491
:1066700011F5F40100935700E89507B600FCFDCF33
:1066800041155105D9F0F60170925700E89537B7DA
:10669000232F217030FDFBCF460110C03091E80060
:1066A0003B7F3093E8003091E80032FDCACF3EB323
:1066B0003111F9CF0FCF41155105D9F2EA01A6CF1B
:1066C0009091F3008091F200892BA1F021976091C5
:1066D000F1008091660190916701DED3809166019F
:1066E00090916701019690936701809366012097CE
:1066F00039F79DCF8091E8008B7F8093E8008091EF
:10670000E80082FDE3CF8EB38111F9CFE3CE809113
:10671000E800877F8093E8008091E80080FF16C042
:10672000809100018930C9F08A30A1F480916D0117
:10673000813081F490916601809167019093F1001E
:106740008093F1008091E8008E7F05CF8EB3811198
:10675000E3CFC0CE80916B01F3CF209166013091E1
:106760006701C0916401D09165012196C21BD30BD2
:1067700080916D01811134C0D695C795C9012091D2
:106780006801A22FB0E0219760F48091640190919C
:106790006501909367018093660182E08093000118
:1067A000D1CF3091F3002091F2002032310559F021
:1067B000FC01259134912093F1003093F100029671
:1067C000A11DB11DE0CF2091E8002E7F2093E800AD
:1067D0002091E80020FDECCF2EB32111F9CF7ACE25
:1067E0008230D9F62097C9F29091F3008091F2009F
:1067F000809791F0809166019091670145D38093D5
:10680000F100809166019091670101969093670174
:10681000809366012197E6CF8091E8008E7F809378
:10682000E8008091E80080FDE5CF8EB38111F9CFBB
:1068300051CE8091E800877F8093E8008091E80046
:1068400080FF11C0809174018093F1001092F100DB
:106850001092F1001092F100809100018093F100FC
:106860001092F1006FCF8EB38111E8CF33CE8091BB
:10687000E800877F8093E800109274016ECE8091CB
:10688000E800877F8093E8008091E80080FF03C0E4
:106890008091000155CF8EB38111F6CF1BCE292FE9
:1068A00030E022303105C9F02330310541F021308C
:1068B0003105C1F090E080E030E020E00AC088239C
:1068C000B1F08130C9F08230A9F782E190E025E093
:1068D00031E0FA013183208308958BE190E027E3D2
:1068E00031E0F7CF82E190E022E531E0F2CF84E0C1
:1068F00090E023E331E0EDCF88E190E029E131E061
:10690000E8CF07B600FCFDCFF999FECF23E0FB01ED
:1069100020935700E89507B600FCFDCF81E18093F6
:106920005700E895089507B600FCFDCFF999FECF12
:1069300025E0FB0120935700E89507B600FCFDCF4A
:1069400081E180935700E895089507B600FCFDCFDC
:10695000F999FECF21E0FB010A0120935700E89549
:106960001124089521E2FC01209357008491089599
:1069700029E0FC01209357008491089589E0E1E02B
:10698000F0E0809357008491089507B600FCFDCF96
:10699000F999FECF809599E0E1E0F0E0082E909320
:1069A0005700E8950895FC0180917F019091800146
:1069B00086179707A0F06115710529F49091E800FA
:1069C0009E7F9093E80090E06115710551F491115C
:1069D00008C08091E80082FF33C080E00895BC01C8
:1069E000F2CF8EB38823B9F18530B9F18091E800F8
:1069F00083FD2FC08091E80082FDEBCF8091E800FD
:106A000080FFE2CF8091F3002091F200382F6115D2
:106A1000710519F02032310558F091E0203231052E
:106A200009F090E02091E8002E7F2093E800CCCF81
:106A300081918093F100615071092F5F3F4FE7CF43
:106A40008EB3882341F0853041F08091E80083FFC8
:106A5000C0CF81E0089582E0089583E00895EBEED1
:106A6000F0E0808181608083EDEEF0E01082609341
:106A7000EC0040838091EE00881F8827881F0895CE
:106A80008091790187FF11C08091E80082FF06C0E4
:106A90008091E8008B7F8093E80003C08EB3811162
:106AA000F3CF08958EB38823E1F38091E80080FF4F
:106AB000F9CF8091E8008E7FEECF62D069D0E0EE12
:106AC000F0E0808181608083E8EDF0E080818F7765
:106AD000808319BCA7EDB0E08C918E7F8C93808170
:106AE0008F7E80831092780108950F931F93CF9328
:106AF000DF9346D04DD0C8EDD0E088818F77888372
:106B000088818068888388818F7D888319BC1EBABC
:106B10001092770100EE10E0F80180818B7F808376
:106B200088818160888342E260E080E098DFE1EE66
:106B3000F0E080818E7F8083E2EEF0E080818160F2
:106B40008083808188608083F80180818E7F80834C
:106B5000888180618883DF91CF911F910F91089583
:106B6000E8EDF0E080818F7E8083E7EDF0E08081CA
:106B70008160808384E082BF81E080937801B5CF1B
:106B8000E8EDF0E080818E7F80831092E20008952E
:106B90001092DA001092E10008951F920F920FB642
:106BA0000F9211242F933F934F935F936F937F9393
:106BB0008F939F93AF93BF93EF93FF938091DA00EE
:106BC00080FF17C08091D80080FF13C08091DA0049
:106BD0008E7F8093DA008091D90080FF88C080E1A9
:106BE00089BD82E189BD09B400FEFDCF81E08EBB85
:106BF00042D18091E10080FF17C08091E20080FFC8
:106C000013C08091E2008E7F8093E2008091E200C9
:106C100080618093E2008091D80080628093D800E8
:106C200019BC85E08EBB27D18091E10084FF29C08B
:106C30008091E20084FF25C080E189BD82E189BDA9
:106C400089B5982F917080FFFBCF8091D8008F7D00
:106C50008093D8008091E1008F7E8093E100809145
:106C6000E2008F7E8093E2008091E2008160809359
:106C7000E20080917701882309F43DC084E08EBB57
:106C8000FAD08091E10083FF21C08091E20083FF70
:106C90001DC08091E100877F8093E10082E08EBB80
:106CA000109277018091E1008E7F8093E1008091C6
:106CB000E2008E7F8093E2008091E2008061809309
:106CC000E20042E260E080E0CADED5D0FF91EF91C1
:106CD000BF91AF919F918F917F916F915F914F91F4
:106CE0003F912F910F900FBE0F901F90189519BCD8
:106CF0001EBAC1D07ECF8091E30087FD93E09EBB9A
:106D0000BFCF1F93CF93DF9300D0CDB7DEB789E716
:106D100091E02091F100FC012193CF01F1E0813855
:106D20009F07B9F7B0DB8091E80083FF0DC0809129
:106D3000790190917A01963009F466C0C8F49923DC
:106D400089F1953009F441C08091E80083FF0AC0C1
:106D50008091E800877F8093E8008091EB0080625B
:106D60008093EB000F900F90DF91CF911F910895CA
:106D7000983009F46BC0993039F78111E5CF9091C3
:106D80007B01923008F78091E800877F8093E800CC
:106D90009093770175DE80917701882309F463C0B1
:106DA00084E066C08D7F803879F68091E800877F27
:106DB0008093E8001092F1001092F1008091E800B9
:106DC0008E7F8093E8005CDEBFCF8111BDCF109134
:106DD0007B011F778091E3008078812B8093E30013
:106DE0008091E800877F8093E8004ADE8091E80088
:106DF00080FFFCCF8091E30080688093E30082E015
:106E0000111183E08EBBA0CF8058823008F09CCF58
:106E100060917D0170917E01AE014F5F5F4F809167
:106E20007B0190917C013BDDBC01892B09F48CCF67
:106E30009091E800977F9093E80089819A81B3DD73
:106E40008091E8008B7F8093E8007ECF803809F046
:106E50007BCF8091E800877F8093E8008091770165
:106E60008093F100ABCF8091E30087FD99CF81E063
:106E70008EBB01D069CF08958EB3882321F0809115
:106E8000E80083FD3ECF0895F999FECF92BD81BD04
:106E9000F89A992780B50895262FF999FECF92BDCB
:106EA00081BDF89A019700B4021639F01FBA20BDCF
:106EB0000FB6F894FA9AF99A0FBE0895F894FFCF96
:106EC000020120DCFB12034C00550046004100206B
:106ED00000440046005500000018034400650061AE
:106EE000006E002000430061006D006500720061CB
:106EF0000000000403090409021B000101008032A4
:106F00000904000000FE0102000921030000000C3A
:106F100010011201100100000020EB03F42F00000B
:046F20000102000169
:107FA0000C9481340C9493340C94A5340C94B23416
:107FB0000C94B8340C94BE340C94C53408950895D0
:067FC000089508950895E4
:107FE000DFCFE0CFE1CFE2CFE3CFE4CFE5CFE6CF05
:087FF000E6CFE6CFE6CFE6CFB5
:087FF8000060000010DFFBDC5B
:040000030000600099
:00000001FF
